:100000000C941E060C9487260C94B4260C94460679
:100010000C9446060C9446060C9446060C94460630
:100020000C9446060C9446060C94D5110C94460686
:100030000C9446060C9446060C9446060C94460610
:100040000C94E1260C9446060C94CF2A0C94122BA7
:100050000C9446060C9446060C9446060C944606F0
:100060000C9446060C9446063017921771177417B5
:1000700077177A177D178017831792178C17C41874
:10008000C618C618C418C618C618C618C618C61882
:10009000C618C618C618C618C618C618C618C61870
:1000A0004A18C618C618C618C618C618BB17C618E8
:1000B000C618C618C618C618C618C618C618C61850
:1000C000C618C618C618C618C618C6185618561820
:1000D0005618561856185618561856185618C61840
:1000E000C618C618C618C618C618BB17551855180E
:1000F00055185518C618631869186F1875187B18A5
:10010000811887188D189718A118AB18B518FC1707
:10011000BE17C618C618C618C6184A18C618C61874
:10012000C618C618C618C618C618C61854185418C3
:1001300054185418C618631869186F1875187B1866
:10014000811887188D189718A118AB18B518FC17C7
:10015000BE17C618C618C618C6184A18F918F918CE
:10016000F918F918F918F918F918F918F918F91807
:10017000F918F918F9180F1A0F1A0F1A0F1A0F1A7F
:100180000F1A3E19481952195C19B919C319D21915
:10019000E3196A1B7F1B8B1B941BA31BC81BD11B62
:1001A0001A1CE31B121F181F1E1F251F331F551F6C
:1001B000731F456E746572206D656E752E2E2E0050
:1001C000546F67676C6564206D6963726F50504D42
:1001D00000546F67676C656420696E76657274653C
:1001E000642050504D2100546F67676C6564205443
:1001F00058206D7574696E672100546F67676C6570
:10020000642074656C656D65747279210050726F3D
:10021000746F636F6C206572726F72207769746897
:100220002052580054696D656F7574207768656E4B
:1002300020636F6E6E656374696E6720746F205201
:100240005800507265737320616E79206B65792058
:10025000746F2063616E63656C00436F6E6E6563DF
:1002600074696E6720746F2052582C20706F776508
:100270007220757020746865205258202877697440
:10028000682062696E6420706C7567206966206EF4
:100290006F74207573696E6720616C776179732064
:1002A00062696E642900546F67676C656420276912
:1002B0006D6D656469617465206F75747075742700
:1002C00000546F67676C65642027736C61766520E6
:1002D0006D6F64652700546F67676C6564202761E4
:1002E0006C776179732062696E642700546F676769
:1002F0006C65642050504D206368616E6E656C20A3
:100300006C696D69740053657420525353492069B8
:100310006E6A656374696F6E206368616E6E656C8A
:100320002028303D3D64697361626C652900536526
:10033000742050504D206D696E696D756D20737914
:100340006E630053657420626561636F6E20696E31
:1003500074657276616C0053657420626561636FC9
:100360006E2064656C617900536574206265616319
:100370006F6E206672657175656E637920696E2097
:10038000487A3A20303D64697361626C652C205074
:10039000783D504D52206368616E6E656C20782CFC
:1003A0002046783D465253206368616E6E656C202E
:1003B00078005365742050574D2073746F7020641B
:1003C000656C61792028302064697361626C6564B2
:1003D0002C20312D323535203D3D20302E317320FB
:1003E0002D2035306D696E29005365742050504DB5
:1003F0002073746F702064656C61792028302064EC
:10040000697361626C65642C20312D323535203D75
:100410003D20302E3173202D2035306D696E29003E
:10042000536574206661696C736166652064656CF0
:1004300061792028302064697361626C65642C20C6
:10044000312D323535203D3D20302E3173202D2089
:1004500035306D696E29002A2A2A2A2A2A2A2A2A50
:100460002A2A2A2A2A2A2A2A2A2A2A2A2A2A2A2AEC
:100470002A2A2A2A0052582041636B6564202D20C5
:1004800072657665727420737563636573736675E0
:100490006C21002A2A2A2A2A2A2A2A2A2A2A2A2AAD
:1004A0002A2A2A2A2A2A2A2A2A2A2A2A2A2A2A2AAC
:1004B000002A2A2A2A2A2A2A2A2A2A2A2A2A2A2AC6
:1004C0002A2A2A2A2A2A2A2A2A2A2A2A2A2A00528E
:1004D000582041636B6564202D20757064617465DC
:1004E000207375636365737366756C21002A2A2A0D
:1004F0002A2A2A2A2A2A2A2A2A2A2A2A2A2A2A2A5C
:100500002A2A2A2A2A2A2A2A2A2A0056616C696457
:100510002063686F69636573206172653A205B319F
:100520005D2D5B31365D20286368616E6E656C20E1
:10053000312D31362900536574206F7574707574D0
:1005400020666F7220706F727420005B585D2061AE
:10055000626F7274206368616E67657320616E6498
:10056000206578697420525820636F6E6669670051
:100570005B535D20736176652073657474696E6783
:100580007320746F205258005B525D20726576654F
:1005900072742052582073657474696E6773207486
:1005A0006F2064656661756C747300557365206EA9
:1005B000756D62657273205B312D445D20746F2010
:1005C0006564697420706F727473205B452D515D92
:1005D00020666F722073657474696E677300202DD6
:1005E00020726563656976657220636F6E66696700
:1005F000757261746F722C20727820737720000AF4
:100600000A6F70656E4C52536E67200053657420FC
:1006100073657269616C2062617564726174653AB8
:10062000200056616C69642063686F696365733A82
:100630002031202D20342B34202F2032202D203823
:10064000202F2033202D20382B34202F2034202D14
:10065000203132202F2035202D2031322B34202FF5
:100660002036202D20313600536574204368616E9A
:100670006E656C20636F6E6669673A20005365741F
:100680002044617461726174652028302D32293AEA
:10069000200053657420486F70206368616E6E653A
:1006A0006C7320286D61782032342C207365706162
:1006B000726174656420627920636F6D6D61732966
:1006C0002076616C69642076616C75657320312DCC
:1006D0003235353A2000536574206368616E6E656B
:1006E0006C2073706163696E6720287831306B48C5
:1006F0007A293A200053657420524620706F77653E
:10070000722028302D37293A200053657420524634
:10071000206D6167696320286865782920652E67E8
:100720002E20307844454144463030443A2000532E
:1007300065742062617365206672657175656E63AC
:10074000792028696E20487A293A20005B5A5D207A
:10075000656E746572207265636569766572206383
:100760006F6E66696775726174696F6E2075746902
:100770006C79005B465D20646973706C61792061FF
:10078000637475616C206672657175656E63696509
:10079000732075736564005B525D2063616C6375E3
:1007A0006C6174652072616E646F6D206B65792079
:1007B000616E6420686F70206C697374005B495DC2
:1007C000207265696E697469616C697A6520736508
:1007D0007474696E677320746F20736B65746368DB
:1007E0002064656661756C7473005B585D2072658A
:1007F00076657274206368616E67657320616E64EC
:100800002065786974206D656E75005B535D20739B
:100810006176652073657474696E677320746F20E8
:10082000454550524F4D20616E64206578697420B3
:100830006D656E7500557365206E756D62657273BA
:10084000205B302D395D20746F20656469742070E1
:100850006172616D657465727300202D2053797328
:1008600074656D20636F6E66696775726174696F18
:100870006E000A0A6F70656E4C52536E672000510D
:1008800029204F7574707574206265666F726520DB
:100890006C696E6B20283D465329203A2000502970
:1008A00020536C617665206D6F64652028657870D3
:1008B0006572696D656E74616C293A20004F29205C
:1008C00054696D65642042494E44206174207374FC
:1008D000617274757020203A20004E292050504DCE
:1008E000206F7574707574206C696D69746564200F
:1008F000202020203A200044495341424C454400E6
:100900004D292050504D205253534920746F20637D
:1009100068616E6E656C202020203A20004C2920F2
:1009200050504D206D696E696D756D2073796E63E1
:10093000202875732920203A200044495341424C15
:100940004544004B29204661696C736166652062ED
:100950006561636F6E20696E74762E2028312D32AA
:10096000353573293A20004A29204661696C736144
:10097000666520626561636F6E2064656C617920D5
:1009800028302D323535203D3E20313073202D204A
:100990003135306D696E293A200049292046616958
:1009A0006C7361666520626561636F6E206672714B
:1009B0002E203A200048292050574D2073746F7024
:1009C0002064656C6179202020202020203A2000BE
:1009D00047292050504D2073746F702064656C61FE
:1009E00079202020202020203A200046292046611E
:1009F000696C736166652064656C617920202020D4
:100A00002020203A200050574D206368616E6E65AB
:100A10006C200066756E6374696F6E3A2000292041
:100A2000706F72742000506F776572546F776572C3
:100A300000445446205548462033322D62697420C4
:100A400031306368004F70656E4C52536E67525878
:100A5000206D696E6920342F36636800466C7974A6
:100A6000726F6E2F4F72616E6765525820554846FF
:100A70002038636800525820747970653A20004429
:100A8000697361626C656400487A00203D3D200016
:100A900043616C63756C61746564207061636B6540
:100AA0007420696E74657276616C3A200042292068
:100AB0004D6963726F202868616C66292050504D23
:100AC000202020203A00412920496E766572746505
:100AD000642050504D20696E20202020203A0030A4
:100AE00029204D7574652062757A7A657220286DAB
:100AF0006F73746C79293A003929205365726961E2
:100B00006C2062617564726174653A00736D617224
:100B100074506F7274004672536B79005472616E38
:100B200073706172656E740044697361626C6564B0
:100B30000038292054656C656D657472793A2020FF
:100B40002020202020003729204368616E6E656CCC
:100B500020636F6E6669673A202000362920446161
:100B60007461726174652028302D32293A2020206A
:100B700000352920486F70206368616E6E656C7364
:100B80003A2020202020003429204368616E6E65C1
:100B90006C2073706163696E673A202000332920EE
:100BA000524620706F7765722028302D37293A2001
:100BB0002020003229205246206D616769633A2067
:100BC0002020202020202020003129204261736530
:100BD000206672657175656E63793A202020000089
:100BE00000000700020100000304060000000000EE
:100BF00000000001020408102040800102040810D7
:100C00002001020408102004040404040404040263
:100C10000202020202030303030303000000002395
:100C2000002600290000000000250028002B0000FD
:100C3000000000240027002A0000002C11241FBE01
:100C4000CFEFD8E0DEBFCDBF13E0A0E0B1E0EEE033
:100C5000FEE502C005900D92AA39B107D9F716E05A
:100C6000AAE9B3E001C01D92AF35B107E1F71CE07E
:100C7000CCE3DCE004C02297FE010E94092DCA33B8
:100C8000D107C9F70E943C2C0C94052F0C9400004E
:100C90008091A505813019F482E08093A5058091AB
:100CA000A505833019F484E08093A5050895A895DF
:100CB0000895DC01ED91FC910190F081E02D099502
:100CC000089561E08AE00E94E42760E08AE00E94E3
:100CD0001D280895892B11F061E001C060E08AE0D1
:100CE0000E941D28089560E08CE00E94E42761E0E6
:100CF0008BE00E94E42761E08DE00E94E42760E041
:100D000082E00E94E42761E084E00E94E4270895E5
:100D100042E050E068E476E080E00E9467260895B3
:100D2000E3E0F0E089E080935700E491E67081E031
:100D3000E63009F080E00895CF93DF93C82F0E943A
:100D40009006882381F0DFB781E08093A405F894B2
:100D50000E94570688E180936000C0936000C11133
:100D60000E945706DFBFDF91CF910895209144057F
:100D700030914505382748E0C901880F991F37FF92
:100D800006C09C0151E2252750E1352701C09C0196
:100D9000415091F730934505209344050895D82F8D
:100DA000C0E0CD1790F45E9A409A64E670E080E06F
:100DB00090E00E945A275E98409864E670E080E0D8
:100DC00090E00E945A27CF5FECCF6CE271E080E0A8
:100DD00090E00E945A27E4CF0F931F93CF93DF93A5
:100DE000EC01062F15E0115051F0CE010E94EC2EBF
:100DF000081741F0602FCE010E94F42EF4CF82E05C
:100E00000E94CF06DF91CF911F910F910895A0E02E
:100E1000B0E0EDE0F7E00C94D22C482E562EC0E066
:100E2000D0E0612C712CE12CF12C00E010E041109D
:100E30000CC06090A30586E4689E30011124A9E1EE
:100E4000EA2EF12C0AE815E01EC091E049120FC00D
:100E50006090A305E6E46E9E30011124FBE16F0E65
:100E6000711CF9E2EF2EF12C06E415E00CC082E0D3
:100E7000481209C078E1672E77247394EE24E39436
:100E8000F12C03EA15E043018C0E9D1E10924505DE
:100E9000109244053401A62CA818B12CC301019668
:100EA0006C01AE14BF04A8F4A00EB11E511006C010
:100EB000C3010E94EC2EF501808305C0F50160811D
:100EC000C3010E94EC06F50180810E94B60636013E
:100ED000E2CFC301511018C0C3010E94EC2EB82EFE
:100EE000C6010E94EC2E2B2D30E0322F2227282B1A
:100EF00080914405909145058217930779F4C0E0ED
:100F0000D0E05524539493CF3601609145050E945B
:100F1000EC0660914405C6010E94EC06C05EDE4FFF
:100F2000C13E92E0D90708F482CF852DCDB7DEB758
:100F3000E0E10C94EE2C87E38093460580E092EC90
:100F4000A1E0B0E08093470590934805A093490540
:100F5000B0934A0587E08093530580E091EAACEBBB
:100F6000B3E380934B0590934C05A0934D05B0934C
:100F70004E0585E0809354058DEE9EEFADEABEED03
:100F800080934F0590935005A0935105B09352055F
:100F9000E5E5F5E080E090E0863028F4DC01AC592E
:100FA000BC4F2C9101C020E021930196883191051E
:100FB00099F782E080936D058AE080936E0508952D
:100FC00061E082E00E940707089560E082E00E94ED
:100FD00007078091A305843020F01092A3050E949A
:100FE000E0070895A1E0B0E0E8EFF7E00C94E02C12
:100FF00089830E94E5079091A3058981981731F0B4
:10100000843020F48093A3050E94E0072196E2E05B
:101010000C94FC2C80E09EECADEEB4E380938B0549
:1010200090938C05A0938D05B0938E0580E090E0A1
:10103000A0E0B0E580938F0590939005A093910573
:10104000B0939205E3E9F5E080E081938F5F803112
:10105000E1F70895A0E0B0E0E0E3F8E00C94D62CCE
:101060000E9437276115710581059105C9F30E941A
:10107000752D10924F051092500510925105109247
:101080005205C4E0C12CD12C7601CA9480904F0542
:1010900090905005A0905105B0905205BA2CA92C03
:1010A000982C88240E94702DA70196010E94B12CD3
:1010B000680D791D8A1D9B1D60934F057093500527
:1010C0008093510590935205C15001F705E515E055
:1010D000E801C12CD12CB2E38B2E912CA12CB12C88
:1010E00080E1E82E87E2F82E8881882309F446C043
:1010F000D39419F40E949B0741C00E94702DA50152
:1011000094010E94B12C21E0260FE5E5F5E08E2F39
:10111000801B8C1520F481918213F9CFE9CF409187
:101120005405249FA00111244E9DC0014F9D900D98
:101130005E9D900D1124AA2797FDA095BA2F40918E
:101140004B0550914C0560914D0570914E05840FF3
:10115000951FA61FB71F40918B0550918C0560917C
:101160008D0570918E05481759076A077B0708F4AB
:10117000BFCF2993C39488E1C812B6CFCDB7DEB7ED
:10118000ECE00C94F22C61E080E00E94070761E043
:1011900081E00E940707089560E080E00E94070751
:1011A000882331F060E081E00E940707811108C0C8
:1011B0000E940A080E949B070E942A080E94C308F6
:1011C00008958436910520F4BC0180E090E017C0BA
:1011D0009C018E3B910528F42A553109AAE0B0E024
:1011E0000CC0823D910528F4245B3109A4E6B0E0EF
:1011F00004C02D5C3109A8E5B2E00E94492CA4E6A8
:10120000B0E09B01AC010E94582C089590E08C59ED
:101210009F4F0E94E10808958F929F92AF92BF92D4
:10122000CF92DF92EF92FF92CF93FC01C0A5EC2FFB
:10123000E770F0E0E45BFC4FA081B0E0C7FF03C0C3
:1012400024E130E002C02FE030E0FC0197A183E10F
:10125000989FF0011124E25CFE4F80809180A28073
:10126000B380A20FB31F20E43FE14DE750E00E949E
:10127000632CA50194010E948F2C8C2F887149F456
:1012800069017A01E0EDCE0EE7E0DE1EE11CF11C03
:101290001BC0C7FF05C060E47AE88CE29EE004C092
:1012A00060E07EEE8AEB9BE069017A01F8EBCF0EFD
:1012B000FBE0DF1EE11CF11CA50194010E948F2CB4
:1012C000C20ED31EE41EF51EC701B60169517C4F44
:1012D0008F4F9F4F28EE33E040E050E00E948F2C6C
:1012E000A8EEB3E00E94582CCF91FF90EF90DF90D2
:1012F000CF90BF90AF909F908F9008958F3F9105B2
:1013000051F048F0811522E0920738F081159340A2
:1013100030F482E0089580E0089581E0089583E04C
:101320000895A0E0B0E0E7E9F9E00C94DB2CEB01D4
:101330008A01B82FB695A0E028813981F801208371
:101340002A813B8121832C813D8122832E813F8113
:101350002383688179814A815B812C813D81EE8183
:10136000FF819F2F9295990F990F907C272F2370C3
:10137000922B252F2370220F220F922B232F2370C5
:101380002295207F922BF80194830B5F1F4F2896A4
:10139000AF5FBA1788F680FF24C0888199810E94C8
:1013A0007E09D82E8A819B810E947E09E82E8C813D
:1013B0009D810E947E09F82E8E819F810E947E0968
:1013C000F0E4DF9EA001112490E1E99E9001112438
:1013D000242B282BE4E0FE9EB0011124262BF801DB
:1013E0002083CDB7DEB7E7E00C94F72C803223E002
:1013F000920708F1883E23E0920740F48F51934012
:10140000E4E096958795EA95E1F70895803D27E019
:10141000920718F48C5D93400895883928E092076C
:1014200068F4885C974074E0969587957A95E1F723
:101430008D509C4F089580E090E008958FEF93E0E9
:1014400008958C30910540F4A4E0880F991FAA9567
:10145000E1F7885D9C4F0895843F23E0920718F4DC
:1014600084529C4F0895811524E0920740F48657DA
:10147000934FF4E0880F991FFA95E1F7089580E9FA
:1014800098E008959C013695279525753575821B42
:10149000930B9C0123733373969587959695879547
:1014A00083739373820F931F9C0154E036952795A5
:1014B0005A95E1F7280F391F2F703F7041E051E036
:1014C000249FC001259F900D349F900D1124892FDA
:1014D00008952D98882319F000002B9A02C000006F
:1014E0002B9800002D9A000008952D9A000083B1DA
:1014F0002D980000829581700895CF93DF93D82FA7
:101500005C9A2D985C98C8E08D2F80780E94690ABB
:10151000DD0FC150C9F72D98DF91CF9108958F77D6
:101520000E947D0A0895CF93DF93D82FC8E08D2FB6
:1015300080780E94690ADD0FC150C9F72D98DF91AC
:10154000CF910895CF93DF932D98C8E080E0D82FF6
:10155000DD0F0E94750A8D0FC150C9F7DF91CF9141
:1015600008950E948F0A0E94A20A5C9A0895A1E041
:10157000B0E0EDEBFAE00C94E02C806869830E9407
:101580007D0A6981862F0E94930A5C9A2196E2E087
:101590000C94FC2CCF93C0914F05C827E82FF0E0A6
:1015A000EA5BFA4F678589E70E94B70A6C2F8DE3E3
:1015B0000E94B70A6C2F82E40E94B70ACF91089567
:1015C00086E20E94B10A0895CF93DF93EC016C810B
:1015D0008CE10E94B70A6D818DE10E94B70A6E818D
:1015E0008EE10E94B70A6F8180E20E94B70A688587
:1015F00081E20E94B70A698582E20E94B70A6A8581
:1016000083E20E94B70A6B8584E20E94B70A6C8568
:1016100085E20E94B70A6D858AE20E94B70A6E854C
:101620008EE60E94B70A6F858FE60E94B70A688926
:1016300080E70E94B70A698981E70E94B70A6A8930
:1016400082E70E94B70ADF91CF910895CF92DF928F
:10165000EF92FF92CF93DF936B017C01C11488E37B
:10166000D8068CE9E8068CE1F80628F5C701B60132
:1016700020E836E948E950E00E948F2CE90168979C
:1016800060E879E687E69FEF0E946B2C6C0D7D1D6C
:101690008E1D9F1DF2E0660F771F881F991FFA9518
:1016A000D1F721E732E040E050E00E948F2CF22E8B
:1016B000E32E80E421C0C701B60120E03DE241E312
:1016C00051E00E948F2CE901689760E073ED8EEC89
:1016D0009EEF0E946B2C6C0D7D1D8E1D9F1D660F55
:1016E000771F881F991F21E732E040E050E00E94F9
:1016F0008F2CF22EE32E80E66C2F6F71680F85E73A
:101700000E94B70A6E2D86E70E94B70A6F2D87E701
:101710000E94B70ADF91CF91FF90EF90DF90CF90BA
:101720000895682F8DE60E94B70A08958F929F92C0
:10173000AF92BF92CF92DF92EF92FF92CF93DF935F
:10174000D82F83E00E94B10A8093430584E00E9471
:10175000B10A8093420560E086E00E94B70A61E02A
:1017600087E00E94B70A6FE789E00E94B70A65E048
:101770008AE00E94B70A62E18BE00E94B70A65E145
:101780008CE00E94B70A6DEF8DE00E94B70A60E01E
:101790008EE00E94B70ADD2319F08BE291E008C0C9
:1017A00020916D0533E1239FC0011124825C9E4F7F
:1017B0000E94E40A6CE880E30E94B70A6FE082E3CB
:1017C0000E94B70A62E483E30E94B70A80916E0523
:1017D00087FF02C064E101C06AE084E30E94B70AA7
:1017E0006AE285E30E94B70A6DE286E30E94B70AC7
:1017F00064ED87E30E94B70A60E088E30E94B70ABD
:1018000060E089E30E94B70AD11109C0C0904F057A
:10181000D0905005E0905105F090520507C0C5E802
:10182000CC2EC1ECDC2EED2CCEEDFC2ECAE38F2CA1
:101830009924AA24BB24682D8C2F0E94B70A682DF6
:1018400085E08C0F0E94B70AFE2CED2CDC2CCC24FA
:10185000CF5FCE3361F76FEF83E40E94B70A6FEF7B
:1018600084E40E94B70A6FEF85E40E94B70A6FEF25
:1018700086E40E94B70ADD2311F066E002C06091A1
:1018800053058DE60E94B70A60E089E70E94B70A17
:10189000609154058AE70E94B70A60E083E70E94DE
:1018A000B70A60E084E70E94B70AD11109C06091CD
:1018B0004B0570914C0580914D0590914E0504C0EB
:1018C00060E071EA8CEB93E30E94260BDF91CF91ED
:1018D000FF90EF90DF90CF90BF90AF909F908F9050
:1018E000089561E087E00E94B70A64E28EE70E94F3
:1018F000B70A63E088E00E94B70A60E088E00E94CF
:10190000B70A65E087E00E94B70A62E085E00E94BE
:10191000B70A83E00E94B10A8093430584E00E94E5
:10192000B10A80934205089583E00E94B10A809332
:10193000430584E00E94B10A8093420561E087E09C
:101940000E94B70A6AE070E080E090E00E945A27A7
:101950000E94710C00000895CF92DF92FF920F93C6
:101960001F93CF93DF931F92CDB7DEB7082F162FAB
:101970008EE399830E94B70AF02EC02E9981D92E4A
:101980008C2D8F19811738F4F60161916F018FE763
:101990000E94B70AF5CF64E085E00E94B70A83E0B1
:1019A0000E94B10A8093430584E00E94B10A8093AB
:1019B00042050E94372760933E0570933F05809350
:1019C00040059093410569E087E00E94B70A81E0F5
:1019D0008093A5050F90DF91CF911F910F91FF90FC
:1019E000DF90CF9008950F931F930E94AC0C8091CD
:1019F000A505813099F40E94372700913E0510918A
:101A00003F052091400530914105601B710B820B11
:101A1000930B603A76488140910548F38091A50583
:101A2000813031F46EE971E083EB95E00E94232967
:101A30001F910F9108950F931F938091A5058230F8
:101A400021F41092A50581E020C08091A505813088
:101A5000D9F40E94372700913E0510913F0520914F
:101A6000400530914105601B710B820B930B613A6D
:101A700076488140910540F061E087E00E94B70A16
:101A80001092A50582E001C080E01F910F9108959A
:101A9000CF93DF93EC014AE050E06D2F70E083EBD1
:101AA00095E00E94F1296EE283EB95E00E94F52813
:101AB000BE0184E0769567958A95E1F76F70772788
:101AC0004AE050E083EB95E00E94F1296EE283EB5F
:101AD00095E00E94F528BE016F7077274AE050E03C
:101AE00083EB95E00E94F129DF91CF91089588233F
:101AF00019F06AEA71E002C06EEA71E083EB95E0EA
:101B00000E9423290895FF920F931F93CF93DF9391
:101B100069EC7BE083EB95E00E94CF2840914B0578
:101B200050914C0560914D0570914E052AE030E0D2
:101B300083EB95E00E94F82963EB7BE083EB95E073
:101B40000E94CF2840914F0550915005609151055A
:101B50007091520520E130E083EB95E00E94F82976
:101B60006DE97BE083EB95E00E94CF284AE050E0EE
:101B70006091530583EB95E00E94202A67E87BE0A3
:101B800083EB95E00E94CF284AE050E06091540535
:101B900083EB95E00E94202A61E77BE083EB95E0F0
:101BA0000E94CF28C5E5D5E0F12C8E0188818823DD
:101BB000A9F0FF2031F061EB71E083EB95E00E942A
:101BC000F22821964AE050E0F801608183EB95E02D
:101BD0000E94E929F394F8E1FF12E7CF83EB95E047
:101BE0000E94FD286BE57BE083EB95E00E94CF2807
:101BF0004AE050E060916D0583EB95E00E94202A59
:101C000066E47BE083EB95E00E94CF28E0916E05CF
:101C1000E770F0E0EE0FFF1FEC5AFC4F608171811E
:101C200083EB95E00E94232961E37BE083EB95E061
:101C30000E94CF2880916E058871883069F028F461
:101C4000811113C068E27BE00CC0803141F0883123
:101C500061F46CE07BE005C06CE17BE002C066E112
:101C60007BE083EB95E00E94112968EF7AE083EB3B
:101C700095E00E94CF28409147055091480560911A
:101C8000490570914A052AE030E083EB95E00E9417
:101C9000F8296FED7AE083EB95E00E94CF288091E0
:101CA0008F0580710E94770D66EC7AE083EB95E0FA
:101CB0000E94CF2880918F0580740E94770D6DEA75
:101CC0007AE083EB95E00E94CF2880918F058072A7
:101CD0000E94770D60E97AE083EB95E00E94CF28BF
:101CE00086E495E00E940C09AB01BC012AE030E0DB
:101CF00083EB95E00E94DA296BE87AE083EB95E0CC
:101D00000E94CF2886E495E00E940C099B01AC015B
:101D100060E472E48FE090E00E948F2CBA01A90188
:101D20002AE030E083EB95E00E94DA2968E87AE067
:101D300083EB95E00E941129CDB7DEB7E5E00C9466
:101D4000F92C8F929F92AF92BF92CF92DF92EF9237
:101D5000FF92811107C06FE77AE083EB95E00E9464
:101D600011292FC090E00E94E10824E630E040E015
:101D700050E00E948F2CCA01B9012AE030E040E017
:101D800050E00E948F2C49015A016B017C012AE02E
:101D900030E0B501A40183EB95E00E94DA296EE200
:101DA00083EB95E00E94F5282AE030E0B701A60118
:101DB00083EB95E00E94DA2963E783EB95E00E94CC
:101DC0003529FF90EF90DF90CF90BF90AF909F901C
:101DD0008F9008951F93CF93DF9365E77AE083EBAD
:101DE00095E00E94CF2880916F05813041F46CE529
:101DF0007AE083EB95E00E94112910E050C0823018
:101E000019F465E47AE0F5CF843019F461E37AE0FF
:101E1000F0CF853091F766E27AE0EBCFC12FD0E0CA
:101E2000C930D1050CF441C068E3610F83EB95E044
:101E30000E94F5286EE17AE083EB95E00E94CF28BE
:101E4000BE016F5F7F4F4AE050E083EB95E00E9458
:101E5000B92963E17AE083EB95E00E94CF28C1596C
:101E6000DA4FE981E03218F566E07AE083EB95E03D
:101E70000E94CF288981803130F06FE373E083EBDB
:101E800095E00E94F22869816F7070E06F5F7F4F6C
:101E90004AE050E083EB95E00E94C2291F5F8091E9
:101EA0001A05181708F4BACF0FC061E3BECFEF7060
:101EB000F0E0EE0FFF1FE659FC4F6081718183EB6C
:101EC00095E00E942329EACF6BEE79E083EB95E061
:101ED0000E94CF28809187050E94A10E60ED79E0D5
:101EE00083EB95E00E94CF28809188050E94A10E87
:101EF00065EB79E083EB95E00E94CF28809189051E
:101F00000E94A10E6AE979E083EB95E00E94CF2858
:101F100040917F0550918005609181057091820507
:101F2000411551056105710539F12AE030E083EB77
:101F300095E00E94F82967E679E083EB95E00E943E
:101F4000CF28809183050E940609AB01BC012AE0DD
:101F500030E083EB95E00E94F82963E479E083EBBD
:101F600095E00E94CF284AE050E06091840583EB21
:101F700095E00E94202A06C06AE379E083EB95E0B1
:101F80000E9411296DE179E083EB95E00E94CF2852
:101F900060918505709186054AE050E083EB95E0FD
:101FA0000E940A2A60E079E083EB95E00E94CF2846
:101FB00060917E05603450F470E06F5F7F4F4AE0BF
:101FC00050E083EB95E00E94C22906C067EF78E0FD
:101FD00083EB95E00E9411296AED78E083EB95E0B0
:101FE0000E94CF2880917D0580FF03C063EB71E0E4
:101FF00002C067EB71E083EB95E00E9423296DEB53
:1020000078E083EB95E00E94CF2880917D05827077
:102010000E94770D6EE978E083EB95E00E94CF286F
:1020200080917D0584700E94770D6FE778E083EBE7
:1020300095E00E94CF2880917D0588700E94770DE1
:10204000DF91CF911F9108950F931F93CF93DF934B
:10205000209117052F3FA9F56FEF75E083EB95E011
:102060000E94CF2884E793E00E94480D6EED75E052
:1020700083EB95E00E94CF28809118059091190577
:102080000E94480D6BEA75E083EB95E00E941129F0
:1020900068E875E083EB95E00E94112960E775E040
:1020A00083EB95E00E9411296BE475E083EB95E0EA
:1020B0000E94112983EB95E00E94FD280E94EA0E00
:1020C00068C012160CF065C0332727FD309580914B
:1020D0001A0590E0821793070CF45BC066E375E085
:1020E00083EB95E00E94CF2860911705772767FD65
:1020F00070954AE050E083EB95E00E94C2296BE0C6
:1021000075E083EB95E00E94CF2810E008E2809113
:102110001B051817D0F5C12FD0E0CC0FDD1FC45E12
:10212000DA4F288130E080911705992787FD909537
:1021300001972817390739F56BEB71E083EB95E0D0
:102140000E94F2284AE050E0602F83EB95E00E9465
:10215000E9296FEB71E083EB95E00E94F228E981B9
:10216000EF70F0E0EE0FFF1FE659FC4F60817181C8
:1021700083EB95E00E94F22863EC71E083EB95E03D
:102180000E94F2280F5F1F5FC2CF83EB95E00E9491
:10219000FD28DF91CF911F910F910895FF920F932A
:1021A0001F93CF93DF93C5E5D5E0F12C8E01888195
:1021B0008823D1F165EC71E083EB95E00E94F22871
:1021C0004AE050E06F2D83EB95E00E94E92962ED33
:1021D00071E083EB95E00E94F2282196F8012081BE
:1021E00030E0A0E1B7E20E94492C9B01AC01A09134
:1021F0005405B0E00E94582CAB01BC0180914B0506
:1022000090914C05A0914D05B0914E05480F591F76
:102210006A1F7B1F2AE030E083EB95E00E94F829DB
:10222000F394F8E1FF12C2CFCDB7DEB7E5E00C942E
:10223000F92C1092B10485E6E2EBF4E0DF011D9287
:102240008A95E9F70895CF93C82F8F3719F0883012
:1022500009F045C0E091B104EE23D9F1E150E093DB
:10226000B104F0E0EE54FB4F10826DE070E083EBC0
:1022700095E00E945906C0E08091B104C81760F44F
:10228000EC2FF0E0EE54FB4F608170E083EB95E0C3
:102290000E945906CF5FF0CF60E270E083EB95E0DB
:1022A0000E9459066DE070E083EB95E00E945906AC
:1022B000C0E08091B104C81778F5EC2FF0E0EE543F
:1022C000FB4F608170E083EB95E00E945906CF5F81
:1022D000F0CF67E083EB95E00E94F5281DC08B31BD
:1022E00019F40E9419111AC08D30C1F08A30B1F072
:1022F0008091B104843668F76C2F70E083EB95E031
:102300000E945906E091B10481E08E0F8093B104E0
:10231000F0E0EE54FB4FC08380E001C081E0CF913C
:102320000895CF93C82F0E94372760939A04709323
:102330009B0480939C0490939D04C093AF04CC2392
:1023400029F040E051EE60E070E004C040E855E262
:1023500060E070E083EB95E00E947F2BCF910895C1
:1023600090919E04492F4F7050E0BA016F5F7F4FEC
:10237000292F30E0E4E035952795EA95E1F76217DB
:10238000730759F0FA01E156FB4F808381E0890F12
:102390008F70907F892B80939E0408956EE770E084
:1023A00083EB95E00E94590608951F920F920FB695
:1023B0000F9211241F932F933F934F935F936F932B
:1023C0007F938F939F93AF93BF93CF93DF93EF93BD
:1023D000FF93C0918600D09187008091590490911D
:1023E0005A0420917B04211155C09E01281B390BF2
:1023F00080918F0590919005A0919105B0919205E3
:1024000085FD02C036952795253C49E03407B8F193
:1024100040910A0150E060E070E01CE1B695A7959C
:10242000979587951A95D1F70097A105B10521F4E5
:1024300081E090E0A0E0B0E084179507A607B70719
:10244000D8F480910A018F3FB9F040E080910A01F1
:10245000481780F4842F90E0880F991FFC01E55AFB
:10246000FB4F20813181FC01E55FFE4F31832083EA
:102470004F5FECCF10927C0410920A010BC02D3BF1
:1024800082E0380720F080910A018031D8F08FEF88
:1024900080930A01D0935A04C0935904FF91EF919D
:1024A000DF91CF91BF91AF919F918F917F916F916C
:1024B0005F914F913F912F911F910F900FBE0F9001
:1024C0001F90189510910A0181E0810F80930A01F5
:1024D000C9010E94F609E12FF0E0EE0FFF1FE55A57
:1024E000FB4F91838083D6CF83E0809380008AE97D
:1024F0008093810080918F0586FD05C080918100C9
:102500008064809381008FEF9FEF90938900809388
:10251000880080916F00806280936F0008956F3013
:1025200018F086958058089589E0689F802D1124C1
:102530000895A0E0B0E0EFE9F2E10C94DA2CC82FA6
:102540000E94372700910A0410910B0420910C047B
:1025500030910D046B017C01C01AD10AE20AF30A22
:102560009701860149E8C41643E1D406E104F10469
:1025700010F010920E0460930A0470930B04809381
:102580000C0490930D0420917B048FEF820F823016
:10259000D8F5E0910E04EE2309F44EC1E13011F4B8
:1025A00082E0B8C1E03108F034C181E08E0F809341
:1025B0000E04F0E0E55AFB4FC083803109F0ACC156
:1025C000EDE5F4E0213029F4A181A695A69580815E
:1025D00008C080819181A92FA695A695A69596956C
:1025E0008795A03148F4B0E090E0AA0FBB1FA55F2B
:1025F000BE4F11969C938E9310927C04329684E089
:10260000EB36F807F9F688C1233009F005C1E091EF
:102610000E04E11104C0CF3009F07EC10DC1E831D4
:1026200048F481E08E0F80930E04F0E0E65AFB4FF1
:10263000C08372C1E83109F0ECC0C111EAC040E0CA
:1026400050E0ABE0CA01B3E0880F991FBA95E1F7FB
:10265000A49F9001A59F300D1124F901E55AFB4F6D
:102660006081E1817E2F777075956795FC01EE0F93
:10267000FF1FE55FFE4F71836083F901E45AFB4F52
:10268000B081B695B695B695E181FE2FF295FF0F14
:10269000F07E6F2F6B2BE695E695E6957E2F777093
:1026A00075956795FC01EE0FFF1FE35FFE4F718389
:1026B0006083F901E35AFB4FB081B295B695B695A8
:1026C000B370C181DC2FDD0FDD0F6D2F6B2BC29539
:1026D000C695C695C370E281E170EE0FEE0F7E2FB6
:1026E0007C2B75956795FC01EE0FFF1FE15FFE4F98
:1026F00071836083F901E15AFB4FB081B695E181A6
:10270000FE2FF795FF27F7956F2F6B2BE6957E2F02
:10271000777075956795FC01EE0FFF1FEF5EFE4F1A
:1027200071836083F901E05AFB4FB081B295BF70AD
:10273000E181FE2FF295F07F6F2F6B2BE295EF700A
:102740007E2F777075956795FC01EE0FFF1FED5E8C
:10275000FE4F71836083F901EF59FB4FB081BB1FBE
:10276000BB27BB1FC181DC2FDD0F6D2F6B2BCC1F57
:10277000CC27CC1FE281E370EE0F7E2F7C2B75956A
:102780006795FC01EE0FFF1FEB5EFE4F71836083C8
:10279000F901ED59FB4FB081B695B695E181FE2F59
:1027A000F295FF0FFF0FF07C6F2F6B2BE695E695F0
:1027B0007E2F777075956795FC01EE0FFF1FE95E20
:1027C000FE4F71836083F901EC59FB4F2081229504
:1027D000269527703181E32FEE0FEE0FEE0F6E2F4F
:1027E000622B732F72957695777075956795FC01BE
:1027F000EE0FFF1FE75EFE4F718360834F5F5F4FF9
:102800004230510509F01ECF8091710483FF109270
:102810007C0410920E0480C0243009F07DC06091C9
:102820000E0461110BC0C83AB1F410924505109224
:10283000440588EA0E94B60681E06CC0613019F454
:10284000C093090404C0623031F4C09308048C2F93
:102850000E94B6065AC0E09108042E2F30E0220FE5
:10286000331F462F50E0C9010296841795073CF0AC
:10287000633268F7FA01E85AFB4FC083E8CF2D5F57
:102880003F4F8C2F90E060914405709145054217B1
:10289000530749F4982F8827862797279093450553
:1028A0008093440532C06817790769F5809109045F
:1028B000813049F5E13118F080E180930804F0900F
:1028C0000804CCE5D4E000E010E00F15D0F4FE01E0
:1028D0003197808190E0982F88272881822B63E0B0
:1028E000969587956A95E1F70E94F609F801EE0F33
:1028F000FF1FE55FFE4F918380830F5F1F4F22967E
:10290000E4CF10927C0410920E0480910E04882370
:1029100019F08F5F80930E04CDB7DEB7E8E00C941A
:10292000F62CE82FF0E0E657FA4FE185E03158F455
:10293000F894F0E0EE0FFF1FE55FFE4F208131813C
:102940007894C9010895E03121F0E13131F483E157
:1029500001C082E10E947928089580E092E0089504
:10296000A2E2B0E0E6EBF4E10C94D02C9E012F5FE4
:102970003F4F80E1D9011D928A95E9F766ED71E03C
:1029800083EB95E029A33AA30E9423290E94940C8B
:102990001D8A1E8A1F8A188E312C212C00E0812C62
:1029A000912C5401412C74E7572E7BE8672E72E37B
:1029B000772EE0E5CE2EE3ECDE2EE12CF12C84EF39
:1029C00091E0A0E0B0E08D8F9E8FAF8FB8A380E044
:1029D0009EECADEEB4E3898F9A8FAB8FBC8F80E015
:1029E00094E7ABE8B2E3898B9A8BAB8BBC8B83EB20
:1029F00095E00E94372A892B09F4E1C083EB95E02A
:102A00000E94642A9C0133272C32310509F442C00C
:102A1000ACF42332310509F0ABC019821A821B8253
:102A20001C821D821E821F82188619861A861B86AA
:102A30001C861D861E861F86188A60C024343105B8
:102A400029F02335310509F4B2C092C064E483EB68
:102A500095E00E94F5282AE030E040E054E76BE87A
:102A600072E383EB95E00E9483296CE283EB95E0AF
:102A70000E94F5282AE030E040E05EEC6DEE74E361
:102A800083EB95E00E9483296CE283EB95E00E9442
:102A90003529ADCF0F5F043009F0A9CF29813A81E4
:102AA0004B815C81A8EEB3E00E94582C698B7A8B35
:102AB0008B8B9C8B2D813E814F8158850E94582C99
:102AC000698F7A8F8B8F9C8F29853A854B855C85A2
:102AD0002D8F3E8F4F8F58A32D853E854F8558896A
:102AE0000E94582C6B017C0160323EE47307810523
:102AF000910530F462E38CE10E94B70A00E077CFE1
:102B0000603345E774078105910510F462E2F3CF65
:102B100060345CE975078105910510F466E2EBCF3E
:102B200080E5C81683ECD806E104F10410F462E1F4
:102B3000E2CF90E6C9169AEED906E104F10410F44A
:102B400065E1D9CFA0E7CA16A1E1DA06A1E0EA065D
:102B5000F10410F461E0CFCFB0EACB16B6E8DB06A3
:102B6000B1E0EB06F10410F463E0C5CF65E0C3CF3C
:102B700010ED180F1A3008F03ACFE1E0F0E0EC0F5A
:102B8000FD1F24E0029FE00DF11D11242081318101
:102B900042815381AAE0B0E00E94582C610F711D60
:102BA000811D911D608371838283938320CF498827
:102BB0005A886B887C88812C912C540118CF811401
:102BC0009104A104B10489F4C301B2010E94260B4F
:102BD00061E070E080E090E00E945A271D8A1E8A22
:102BE0001F8A188E312C22242A948D8D9E8DAF8DB4
:102BF000B8A188169906AA06BB06D0F40E94E00A7E
:102C00002D893E894F89588D280F311D411D511D39
:102C10002D8B3E8B4F8B588F381608F4382E82152B
:102C200008F4282E3FEF831A930AA30AB30A56C06A
:102C3000C301B20128EE33E040E050E00E948F2C47
:102C4000BA01A9012AE030E083EB95E00E94DA297D
:102C50006CE283EB95E00E94F5284AE050E0632D9A
:102C600083EB95E00E94E9296CE283EB95E00E94FA
:102C7000F5286D897E898F89988DA50194010E9420
:102C80008F2CBA01A9012AE030E083EB95E00E9485
:102C9000DA296CE283EB95E00E94F5284AE050E0E7
:102CA000622D83EB95E00E94E9296CE283EB95E0CD
:102CB0000E9435294C0C5D1C6E1C7F1C898D9A8DE1
:102CC000AB8DBC8D84159505A605B70520F4498804
:102CD0005A886B887C88812C912C540129893A89E7
:102CE0004B895C89283E33404105510509F07FCE70
:102CF000A296E2E10C94EC2CACE1B0E0E2E8F6E163
:102D00000C94DA2C0E9437276B017C0181E00E9431
:102D1000960B14E703E0198361E0CE0101960E944F
:102D2000F30C0093A5050E94710C6AEF70E080E03F
:102D300090E00E945A278091A505833089F483EBA7
:102D400095E00E94372A892B59F40E9437276C1985
:102D50007D098E099F096038734C894C9140D8F2E7
:102D60008091A505833009F44FC08FE70E948F0A38
:102D70000E94A20A8983843511F083E05CC00E941E
:102D8000A20A10921805809319050E94A20A2091A8
:102D9000180530911905280F311D3093190520931E
:102DA00018050E94A20A80931A050E94A20A809325
:102DB0001B05813110F7F12C0F2D10E080911B05C0
:102DC00090E0880F991F0817190740F40E94A20A83
:102DD000F801E45EFA4F8083F394EECF80E78983B5
:102DE00061E0CE0101960E94F30C83E08093A5057B
:102DF0000E94710C62E370E080E090E00E945A272C
:102E00008091A505833011F482E015C08FE70E9400
:102E10008F0A0E94A20A8983803509F0AECF0FE69F
:102E200015E00E94A20AF80181938F01F5E00A38AB
:102E30001F07B9F781E06C96E8E00C94F62C8091BE
:102E40001705992787FD9095A92FB92FFC01319679
:102E5000EB30F10508F066C0EC5CFF4F0C94072DD9
:102E600062E778E083EB95E00E94112984E793E024
:102E70000E94480D6AE578E083EB95E00E941129F5
:102E800065E378E083EB95E00E9411296BE078E040
:102E900083EB95E00E9411296AEE77E083EB95E0E1
:102EA0000E9411296DEB77E083EB95E00E941129D8
:102EB00067E977E083EB95E00E94112963E777E00B
:102EC00083EB95E00E9411296CE477E083EB95E0B9
:102ED0000E94112983EB95E00E94FD280E94830D3A
:102EE00021C06FE277E01AC06AE077E017C065EFB3
:102EF00076E014C066ED76E011C062E976E00EC0BF
:102F00006DE776E00BC068E676E083EB95E00E9423
:102F1000112962E276E002C06CE076E083EB95E096
:102F20000E9411296AE070E080E090E00E945A2738
:102F300083EB95E00E94372A892B29F083EB95E0FB
:102F40000E94642AF5CF0895ACE1B0E0EAEAF7E127
:102F50000C94DA2C909117059F3F09F023C1482F5C
:102F600050E0FA013A97EF36F10508F00FC1E15C45
:102F7000FF4F0C94072D63EE71E0A0C06FEE71E07F
:102F800083EB95E00E94232985E789838BE1EFE6B7
:102F9000F5E0DE01129601900D928A95E1F76CE161
:102FA000CE0101960E94F30C0E94710C83E0809385
:102FB000A50568EC70E080E090E00E945A278091BF
:102FC000A505843009F0E2C08FE70E948F0A0E94B5
:102FD000A20A8983853509F0D9C06DEE74E083EBD0
:102FE00095E00E9411296FEC74E083EB95E00E945C
:102FF000112961EB74E096C067E072E083EB95E025
:103000000E94232989E6898361E0CE0101960E940E
:10301000F30C0E94710C83E08093A50568EC70E0CE
:1030200080E090E00E945A278091A505843009F045
:10303000ADC08FE70E948F0A0E94A20A89838E0189
:103040000E5F1F4F7E014DE1E40EF11C0E94A20AAB
:10305000F80181938F01EE15FF05C1F78BE1FE01A9
:103060003296AFE6B5E001900D928A95E1F789813D
:10307000893409F08BC063E974E083EB95E00E942A
:10308000112965E774E083EB95E00E94112967E55B
:1030900074E048C061E272E083EB95E00E9423296E
:1030A0008EEF8093170572C08052875080539091A5
:1030B0001A05981708F066C060E372E083EB95E0AC
:1030C0000E94232963C084E18093170560E274E0C5
:1030D00029C085E18093170569EE73E023C086E17E
:1030E0008093170562EB73E01DC087E1809317059D
:1030F00068E673E017C088E18093170567E573E021
:1031000011C089E18093170563E473E00BC08AE185
:10311000809317056EE273E005C08BE1809317057D
:1031200066E073E083EB95E00E9411292FC06CEEFE
:1031300072E083EB95E00E94112980917D0591E07A
:103140001DC066ED72E083EB95E00E94112980912D
:103150007D0592E013C061EC72E083EB95E00E9484
:10316000112980917D0594E009C066EA72E083EB45
:1031700095E00E94112980917D0598E08927809330
:103180007D058FEF809317050E94241083EB95E057
:103190000E94372A892B09F45AC183EB95E00E94DB
:1031A000642AF4CF0E942311882309F450C180912E
:1031B000B104811104C08FEF8093170540C140E036
:1031C00050E060E070E082EB94E00E947E2D409140
:1031D0001705042F112707FD1095212F312FF80116
:1031E0003197EB31F10508F01AC1E255FF4F0C940D
:1031F000072D552747FD509520911A0530E02417DB
:1032000035070CF40CC18B019C01015011092109F7
:103210003109003211052105310558F0C0901B0518
:10322000EDE1F5E0F12CD12CA8E2EA2E4150510954
:103230000FC0FA01E159FA4F61506083D8C0DF0135
:1032400011972C9130E02417350729F0F39432962A
:10325000FC10F5CFCAC00E2D10E020E030E00617BC
:1032600017072807390741F42081DA01A159BA4F1D
:1032700011962C93DD24D394E394E8CF6F3F71052E
:103280008105910511F008F0CAC060938705AFC0B1
:103290006F3F71058105910511F008F0C0C0609382
:1032A0008805A5C06F3F71058105910511F008F0F3
:1032B000B6C0609389059BC02091B204206220377C
:1032C000E9F440E050E060E070E083EB94E00E94BD
:1032D0007E2D9B01AC01DC01CB010197A109B10955
:1032E0000897A105B10508F0ADC0A4EDB0E30E94B8
:1032F000582C6A5E7C4A8A46954E24C02636E9F4EC
:1033000040E050E060E070E083EB94E00E947E2DAE
:103310009B01AC01DC01CB010197A109B109079721
:10332000A105B10508F08EC0A8EAB1E60E94582CAC
:10333000645E7C438E46944E05C06115710581051F
:10334000910571F08B019C0114572B4832430130D9
:10335000FAE51F07F2E62F07F2E03F0708F05FC02B
:1033600060937F057093800580938105909382051B
:103370003EC06F3F71058105910511F008F04FC007
:103380006093830534C08B019C0101501109210910
:1033900031090F3F11052105310508F040C0609348
:1033A000840525C08B019C01045C19402109310969
:1033B0000D344DE114072105310528F4709386057D
:1033C0006093850514C0611571058105910521F48F
:1033D0008FEF80937E050BC06134710581059105E7
:1033E000F0F4615060937E0502C0DD20C1F0809151
:1033F000B00481111AC080914F0590915005A091A1
:103400005105B09152050196A11DB11D80934F0544
:1034100090935005A0935105B093520506C062E405
:1034200072E083EB95E00E9423290E9419118FEF2F
:10343000809317056AE083EB95E00E9435290E948E
:10344000241005C061E070E080E090E07BCF6C96D6
:10345000E8E00C94F62C6AE572E083EB95E00E94BC
:10346000112962E472E083EB95E00E94112983EB5D
:1034700095E00E94372A892B31F083EB95E00E947A
:10348000642A0E94A4170E947C16823029F083309F
:1034900051F46DE072E002C064E272E083EB95E00B
:1034A0000E94112908958FEF809317051092B004A0
:1034B0000E942410809117058E3F69F083EB95E000
:1034C0000E94372A892BB1F383EB95E00E94642A8E
:1034D0000E94A417EFCF08950F931F931091170523
:1034E0001F3F09F0D1C0893409F457C000F5883373
:1034F00009F468C058F4803309F476C008F060C05D
:103500008B3109F440C08132B1F1B8C0813409F483
:1035100086C030F4893309F465C0803461F1AEC0EF
:10352000823409F48DC0863409F447C0A7C08236BE
:1035300009F486C078F4883531F128F48235C1F178
:103540008335E1F09BC08A3509F493C0813609F4D4
:1035500066C094C0823761F128F4863671F18936ED
:10356000E1F08CC0883779F08A3709F482C083375C
:1035700009F084C003C063EE71E015C00E94C30867
:1035800060E672E004C00E94CC086AE772E083EB58
:1035900095E00E9423298EEF6FC00E949B070E9436
:1035A0000A0869E972E083EB95E00E94232966C06E
:1035B0000E942A0862EB72E0F6CF0E94CE105EC035
:1035C00080535AC06AEF71E083EB95E00E941129A5
:1035D00090916E0588E0890F8871977E892B809382
:1035E0006E051AC089E048C067EE71E083EB95E094
:1035F0000E94112980918F0590919005A0919105CD
:10360000B091920520E1822780938F0590939005D9
:10361000A0939105B0939205109317052FC061ED0B
:1036200071E083EB95E00E94112980918F059091C4
:103630009005A0919105B091920540E4842710C0B7
:1036400060EC71E083EB95E00E94112980918F0579
:1036500090919005A0919105B091920520E282276A
:1036600080938F0590939005A0939105B093920558
:1036700002C00E942B1A8FEF8093170580911705C7
:103680008E3F09F0D4C0DDC00E942311882309F4C5
:10369000D8C08091B104811104C08FEF80931705C9
:1036A000C6C040E050E060E070E082EB94E00E9431
:1036B0007E2D00911705112707FD1095212F312F21
:1036C000F8013197E930F10508F0B4C0E753FF4F36
:1036D0000C94072D8B019C01015014472B48324359
:1036E0000F3F19452246324008F0A4C060934B05B5
:1036F00070934C0580934D0590934E0577C0609371
:103700004F0570935005809351059093520581E0C9
:103710008093B0046BC0683071058105910508F095
:1037200089C06093530562C08B019C01015011094F
:10373000210931090A3011052105310508F07AC047
:103740006093540553C061EB71E082EB94E00E94FA
:10375000B82E10E0009799F00E94922E009779F011
:10376000183130F4E12FF0E0EA5BFA4F87871F5FF2
:1037700061EB71E080E090E00E94B82EEBCF183151
:10378000A8F5E12FF0E0EA5BFA4F17861F5FF7CF4D
:10379000653071058105910508F04CC060936D0599
:1037A00025C08B019C010150110921093109063006
:1037B000110521053105F0F520916E05287F262B96
:1037C00020936E0513C08B019C0101501109210942
:1037D00031090115124C2140310560F56093470510
:1037E000709348058093490590934A058091B004F1
:1037F000811113C080914F0590915005A091510502
:10380000B09152050196A11DB11D80934F05909373
:103810005005A0935105B09352050E9419118FEFE6
:10382000809317056AE083EB95E00E9435290E949A
:103830001F1707C062E472E083EB95E00E94232922
:10384000ECCF1F910F9108958FEF80931705109281
:10385000B0040E941F17809117058E3F69F083EB1B
:1038600095E00E94372A892BB1F383EB95E00E9403
:10387000642A0E946C1AEFCF6AE070E080E090E06A
:103880000E945A2783EB95E00E94372A892B29F062
:1038900083EB95E00E94642AF5CF0895CF93C82F5B
:1038A000682F83EB95E00E94912A90913C059C271C
:1038B00090933C05CF910895A1E0B0E0E2E6FCE1F1
:1038C0000C94E02C99830E944E1C9981892F0E94B0
:1038D0004E1C2196E2E00C94FC2C1F93CF93DF93B7
:1038E000182FEB0110923C0565EB70E083EB95E03F
:1038F0000E94590662E670E083EB95E00E9459064B
:10390000812F0E944E1CCE010E945C1CDF91CF9142
:103910001F91089560913C0583EB95E00E94912AE8
:103920000895A1E2B0E0E7E9FCE10C94DC2C7B0116
:103930008A018B3009F42EC108F03FC0853009F4AC
:103940009BC010F5823009F47EC058F4813009F034
:1039500030C269E270E081E00E946D1C06E415E06F
:1039600068C0833009F480C0843009F022C261E06D
:1039700070E084E00E946D1C81E00E944E1C0E9459
:103980008A1C0E94B0141FC2883009F49BC070F4D6
:10399000863009F48DC0873009F00BC261E070E019
:1039A00087E00E946D1C80911A0509C2893009F4D4
:1039B00091C08A3009F4C3C0FCC1893609F469C1D9
:1039C00078F4863609F41AC120F4853609F402C168
:1039D000F0C1873609F426C1883609F42BC1E9C144
:1039E0008C3609F49FC190F48A3609F45CC18B3699
:1039F00009F0DFC161E070E08BE60E946D1CF80108
:103A000080810E94F2070E94CC08BEC18D3609F465
:103A1000BDC1873C09F0CDC161E070E087EC0E9438
:103A20006D1C81E00E944E1C0E948A1C10923D0574
:103A3000CAC1F80181918F010E944E1CF5E00F363A
:103A40001F07B9F7BEC16BE170E082E00E946D1CF8
:103A50000FE615E0F80181918F010E944E1CF5E000
:103A60000A381F07B9F7ADC161E070E083E00E943A
:103A70006D1C0E947C16A3C160911B0570E0660F4F
:103A8000771F85E00E946D1C0CE115E080911B05FD
:103A900090E0880F991F98012C513540281739075D
:103AA00008F08FC1F80181918F010E944E1CEECF6A
:103AB00062E070E086E00E946D1C84E793E00E9463
:103AC0005C1C7FC161E070E088E00E946D1C809109
:103AD000A30575C186E6898361E0CE0101960E9447
:103AE000F30C0E94710C83E08093A50568EC70E0F4
:103AF00080E090E00E945A278091A5058430D9F497
:103B00008FE70E948F0A0E94A20A8983863469F493
:103B100060E270E089E00E946D1C10E20E94A20A3F
:103B20000E944E1C1150D1F74CC161E070E089E059
:103B30000E946D1C29C161E070E089E03DC169E12E
:103B400070E08AE00E946D1C81E080938A052091DC
:103B5000A40580918F0590919005A0919105B09159
:103B60009205222311F0806801C08F7780938F0522
:103B700090939005A0939105B09392050AE815E003
:103B8000F80181918F010E944E1CF5E0033A1F0756
:103B9000B9F717C161E270E08BE00E946D1C809163
:103BA0007C048F3F39F080917C0491E0980F9093D2
:103BB0007C0402C080917C040E944E1C10E0812F86
:103BC0000E9491140E94210A0E945C1C1F5F103108
:103BD000B1F7F7C061E070E085E60E946D1C89E2F4
:103BE000E816F10409F0EAC0D801E6E4F5E08D91A9
:103BF000819385E0EF36F807D1F7C6C061E070E049
:103C000086E60E946D1CEBE1EE16F10409F0D6C0C9
:103C1000D801EFE6F5E08D91819385E0EA38F80769
:103C2000D1F7B2C061E070E087E60E946D1C0E948F
:103C3000C308AAC061E070E088E60E946D1C85E7B9
:103C400089838BE1EFE6F5E0DE01129601900D929B
:103C50008A95E1F76CE1CE0101960E94F30C0E9477
:103C6000710C83E08093A50560E273E080E090E052
:103C70000E945A278091A505843009F09FC08FE7E4
:103C80000E948F0A0E94A20A8983853509F096C096
:103C90007BC061E070E089E60E946D1C0E949B077A
:103CA0000E940A0871C061E070E08AE60E946D1C03
:103CB00089E6898361E0CE0101960E94F30C0E949F
:103CC000710C83E08093A50560E273E080E090E0F2
:103CD0000E945A278091A505843009F06FC08FE7B4
:103CE0000E948F0A0E94A20A89838E010E5F1F4FD5
:103CF0007E01EDE1EE0EF11C0E94A20AF801819313
:103D00008F01EE15FF05C1F78BE1FE013296AFE69C
:103D1000B5E001900D928A95E1F78981893409F027
:103D20004DC032C061E070E08CE60E946D1CF0E294
:103D3000EF16F10461F487E6898380E2F801DE0181
:103D4000129601900D928A95E1F761E203C087E433
:103D5000898361E0CE0101960E94F30C0E94710CF0
:103D600083E08093A5056CE474E080E090E00E941D
:103D70005A278091A505843009F58FE70E948F0AA4
:103D80000E94A20A8734D1F481E019C061E070E09A
:103D90008DE60E946D1C89E1E816F10479F4D801E2
:103DA000EAE8F5E08D91819385E0E33AF807D1F7F1
:103DB000EBCF61E070E08AEC0E946D1C80E00E9415
:103DC0004E1C0E948A1CA196E6E00C94F82CA0E000
:103DD000B0E0EDEEFEE10C94DA2CCCE9D3E014E691
:103DE00006E035E0F32E44E0E42E53E0D52E62E009
:103DF000C62E83EB95E00E94372A892B09F49BC0DD
:103E000083EB95E00E94642A282F80930704409159
:103E1000060450E04730510560F7FA01EE52FF4FBB
:103E20000C94072D853B29F781E080930604E1CFB0
:103E3000823609F07DC0C0920604DBCF8093050472
:103E400080930404D0920604D4CF9C01332730938E
:103E5000030420930204909104049827909304048F
:103E6000E0920604C6CF382F2227409102045091D9
:103E70000304242B352B30930304209302049091E8
:103E80000404982790930404F09206042536310523
:103E900008F4AFCF61E070E08CEC0E946D1C81E013
:103EA0000E944E1C0E948A1C43C020910004309145
:103EB0000104F901E456FC4F808390910404982793
:103EC00090930404C9010196909301048093000427
:103ED00020910204309103048217930708F489CFDC
:103EE0000093060486CF8091040482130BC0609176
:103EF0000004709101044CE953E0809105040E9494
:103F0000911C0DC062E070E08BEC0E946D1C8091F2
:103F100005040E944E1C80913C050E944E1CFE012F
:103F2000812F11928A95E9F71092010410920004F2
:103F3000109206045ECFCDB7DEB7E8E00C94F62C05
:103F400081E080933D0580913D05882349F083EB16
:103F500095E00E94372A892BB1F30E94E71EF3CF28
:103F60000895AAE2B0E0E7EBFFE10C94D82C0E94A0
:103F70002B276B017C0181E00E94960B83EB95E07F
:103F80000E94372A892B29F083EB95E00E94642A4E
:103F9000F5CF5E98409811E072E6B72EE9E2AE2EBA
:103FA00003E00E942B276C197D098E099F09693C4B
:103FB000710581059105E0F11123D1F10E942B27B4
:103FC0006B017C015D9A419A80ED97E00E946A0640
:103FD000B982E6E4F5E0DE0112968A2D01900D9299
:103FE0008A95E1F76AE2CE0101960E94F30C5D9892
:103FF000419880E090E00E946A060093A5050E9427
:10400000710C62E370E080E090E00E945A2780919A
:10401000A505843061F40093A5058FE70E948F0AFF
:104020000E94A20A11E0823419F410E001C011E0EC
:1040300083E10E945028892BA1F411E012C05E9AFE
:10404000409A5D9A419A83EB95E00E94642A8D30F4
:104050009105B9F06CF40A97A1F05E9840985D98CC
:10406000419883EB95E00E94372A892B41F799CF3D
:104070008332910579F08234910579F70E94A01F6F
:10408000ECCF62EB71E083EB95E00E9411290E9476
:10409000241CE3CF0E94B014E0CF8F929F92AF9286
:1040A000BF92CF92DF92EF92FF921F93CF93DF9355
:1040B00083E10E945028892B09F078C068EC70E0F9
:1040C00080E090E00E945A2780E090E00E946A061B
:1040D0000E942B274B015C016B017C0180ECC80E18
:1040E00082E1D81EE11CF11C0E942B276C157D0576
:1040F0008E059F0530F483E10E945028892BA1F39F
:1041000053C083E10E945028892B09F04DC080EDF7
:1041100097E00E946A060E942B276B017C01D0E089
:10412000C1E088E4880E86E2981EA11CB11C11E053
:1041300083E10E945028892B21F58C149D04AE0444
:10414000BF0430F480ED97E00E946A06D1E0F0CF22
:104150000E942B276C197D098E099F09693C710506
:104160008105910528F30E942B276B017C01C12753
:1041700019F080ED97E002C080E090E00E946A06AE
:10418000D7CF80E090E00E946A06DD2349F080915D
:10419000A3058F5F83700E94F2070E94CC0806C0BF
:1041A0000E942A080E94C3080E94B11FDF91CF918C
:1041B0001F91FF90EF90DF90CF90BF90AF909F90B6
:1041C0008F900895CF92DF92EF92FF9280E00E944D
:1041D0009C060E94730661E086E00E94E42761E08D
:1041E00085E00E94E42761E08EE00E94E42761E020
:1041F0008FE00E94E42760E083E10E94E42760E012
:1042000088E00E94E42761E088E00E941D280E9467
:10421000610640E052EC61E070E083EB95E00E94C3
:104220007F2B0E94E5070E94CC080E9474128FEF3A
:1042300080937C040E94880678940E942B276B014F
:104240007C0180917C048F3F59F40E942B276C19CC
:104250007D098E099F09603D77408105910588F3AE
:1042600080ED97E00E946A0661E083E10E941D28CC
:104270005E9A409A83EB95E00E94372A892B29F0B9
:1042800083EB95E00E94642AF5CF6FEC72E083EB3C
:1042900095E00E94F22884E793E00E94480D66EEC4
:1042A00072E083EB95E00E94F2284AE050E069E07A
:1042B00070E083EB95E00E94C22962E370E080E049
:1042C00090E00E945A2783EB95E00E94372A0497DA
:1042D0000CF183EB95E00E94642A82349105D1F4BD
:1042E00083EB95E00E94642A8E34910599F483EB68
:1042F00095E00E94642A8434910561F483EB95E093
:104300000E94642A819731F480E090E00E946A065E
:104310000E94B11F409147055091480560914905A1
:1043200070914A05DB01CA010197A109B1090497FF
:10433000A105B10568F440937B04433029F440EAB9
:1043400056E861E070E004C040E052EC61E070E0EB
:1043500083EB95E00E947F2B0E944D205E98409851
:1043600080E090E00E946A060E9474121092970406
:1043700080918F0583FF11C080915B05882351F0E8
:1043800080916205882331F080916905882311F0BE
:1043900087E001C085E08093970480E00E94960B3F
:1043A000809198040E94CA0A0E94710C1092110414
:1043B0001092100410920F04F12C8091A3058F1518
:1043C000B0F062E370E080E090E00E945A2780ED58
:1043D00097E00E946A0662E370E080E090E00E944D
:1043E0005A2780E090E00E946A06F394E6CF80911D
:1043F0006E0584FF08C0982F987181E0983109F00C
:1044000080E00E9491118FE00E949C06FF90EF9047
:10441000DF90CF900895EF92FF920F931F93CF9369
:10442000DF938C016EE770E083EB95E00E94590604
:10443000E801F12CF0E2EF2E8E0188818D57823059
:1044400048F46DE770E083EB95E00E94590688819F
:104450008E2588832196F801608183EB95E00E9488
:10446000912AF394F9E0FF12E7CF6EE770E083EB57
:1044700095E00E945906CDB7DEB7E6E00C94F82C23
:10448000A9E0B0E0E6E4F2E20C94E02C909199040B
:1044900091110EC09EEF99838A836B8350E05595EE
:1044A00047954C832D83198618861F821E822EC045
:1044B00040919E04842F90E0B4E095958795BA953D
:1044C000E1F7242F2F7030E08217930719F18DEF59
:1044D00089831B82FE01349650E0842F90E0A4E093
:1044E00095958795AA95E1F7242F2F7030E08217D4
:1044F000930749F0DC01A156BB4F8C918193405F3B
:104500005F5F563051F740939E045A83CE01019667
:104510000E940B228091990490E0019666E070E081
:104520000E947B2C809399042996E2E00C94FC2C49
:10453000A0E0B0E0EEE9F2E20C94D92C6C016EE759
:1045400070E083EB95E00E9459068601E12CF12C86
:10455000C0E0D0E030E2B32EF801608183E8860F3E
:10456000823078F46DE770E083EB95E00E945906A5
:10457000F80160816B2570E083EB95E00E9459069D
:1045800004C083EB95E00E94912AE114F10459F0F4
:10459000F80180819E01280F311DC901C92FDD2737
:1045A000C80FD91FDD273FEFE31AF30A89E0E816A9
:1045B000F10459F028E0E216F10421F48C2F8095E3
:1045C000F60180870F5F1F4FC7CFCDB7DEB7E9E099
:1045D0000C94F52CA9E0B0E0E0EFF2E20C94E02CB2
:1045E000E82F362F8091990490E0019664E270E004
:1045F0000E947B2C8093990458E9598350E15A8397
:10460000813089F048F08230B9F08330D9F48B835F
:1046100081EF8C833D8319C085E08B8381EF8C8390
:104620002F5F2D8312C08B8381EF8C8384E6489F9C
:10463000A00111245D8309C084E08B8381EF8C830A
:10464000ED8303C00E94CE1104C0CE0101960E94EA
:1046500098222996E2E00C94FC2CA2E0B0E0E3E37F
:10466000F3E20C94D52C182F762E2A8349830E94CE
:1046700037276B017C018091AF0480909A04909061
:104680009B04A0909C04B0909D042A8149818823BA
:10469000C1F0D701C60188199909AA09BB094C01C3
:1046A0005D0191EE89169EE29906A104B10420F104
:1046B000241708F4422F202F672D812F0E94EA2211
:1046C00013C0D701C60188199909AA09BB094C0171
:1046D0005D0191E3891695E79906A104B10460F0A4
:1046E000672D812F0E944022C0929A04D0929B0491
:1046F000E0929C04F0929D042296EDE00C94F12C43
:10470000A2E2B0E0E6E8F3E20C94D62C8CE00E9442
:10471000B10A81110FC06EEE72E083EB95E00E944A
:1047200023295E9A409A80E00E94960B0E94710CA9
:104730005E98409883EB95E00E94372A892B01F11F
:1047400083EB95E00E94642A90917B04992319F0F1
:104750000E949912EFCF4091100450E09A012F5F10
:104760003F4F2F7133276091110470E026173707F0
:1047700009F3FA01E55EFB4F808320931004DACF42
:104780008091A505843009F086C00E943727611505
:1047900071058105910549F06093890470938A043D
:1047A00080938B0490938C040CC081E090E0A0E097
:1047B000B0E08093890490938A04A0938B04B09313
:1047C0008C0480917F049091800481609093800498
:1047D00080937F0483E08093A5058FE70E948F0A72
:1047E0000BE314E00E94A20AF80181938F01F4E028
:1047F00004341F07B9F72091440480913B04982F9B
:10480000922796FF3BC090E4922790934404982F00
:1048100098739833F1F410E0212F30E080913B043D
:10482000877090E0821793074CF11F5F20916E050F
:10483000812F90E0FC01E55CFB4F24FF04C08081E8
:104840000E94B011E9CF608183EB95E00E94912A2C
:10485000E3CF8F7399F480913C0480938804809116
:104860003D048093860480913E048093850480916A
:10487000410490E090937E0480937D0480910F0426
:10488000813019F482E080930F0480910F0483300B
:1048900011F410920F040E9437276B017C01809164
:1048A000810490918204A0918304B09184040097C4
:1048B000A105B105C9F0A7019601281B390B4A0BC8
:1048C0005B0BDA01C901883B9B40A105B10560F093
:1048D0000E94E00A8093870410928104109282045F
:1048E000109283041092840480918D0490918E0420
:1048F000A0918F04B091900446015701881A990A3B
:10490000AA0ABB0A86E495E00E940C09861697065F
:10491000A806B90608F4A5C0C0928D04D0928E04F2
:10492000E0928F04F09290040E94570680917C04DC
:104930008830A0F080918F0590919005A09191050D
:10494000B09192056CE1B695A795979587956A9574
:10495000D1F7892B8A2B8B2B09F0ABC180917C047A
:104960008F5F80937C048091890490918A04A09148
:104970008B04B0918C040097A105B105F1F0C81A21
:10498000D90AEA0AFB0A86E495E00E940C096C1534
:104990007D058E059F0508F004C180918F0584FD7B
:1049A00004C080ED97E00E946A061092890410927C
:1049B0008A0410928B0410928C0490914404907C91
:1049C00090934404509110048091110420910F049D
:1049D000581709F403C1223009F000C19058909390
:1049E0004404E0916E05E770F0E0E45BFC4F608109
:1049F000693008F0DBC0615040E04613D9C08093B5
:104A0000110487E3840F90914404892B809344041C
:104A10004093120483E080930F045D9A419A909131
:104A20009704911130C1809198040E94CA0AE091C4
:104A30006E05E770F0E0E45BFC4F608184E494E095
:104A40000E94AC0CE0919804EF5FE0939804E83189
:104A500009F42CC1F0E0EA5BFA4F8785882309F45A
:104A600025C10E941B0D813069F580916E0588710A
:104A700049F180917F0490918004880F991F909351
:104A8000800480937F0483E08093A5050E94710CCD
:104A90000E9437276093810470938204809383047B
:104AA00090938404672B682B692B61F481E090E07C
:104AB000A0E0B0E08093810490938204A0938304EB
:104AC000B093840480916E0584FF1FC080917F04A1
:104AD000909180048E7F0E94420A182F60917D047D
:104AE000809188040E948F12482F612F8091870443
:104AF00049A30E948F120091A305282F49A160911C
:104B00008504809186040E942D235D9841988091B0
:104B100095048130C1F018F08230B1F1D4C083E146
:104B20000E945028892B09F0CEC081E08093950423
:104B30000E942B27609391047093920480939304B6
:104B400090939404C0C083E10E945028892B31F5D2
:104B50000E942B27C0909104D0909204E09093047F
:104B6000F09094046C197D098E099F09693E734089
:104B70008105910508F4A7C082E08093950480ED3B
:104B800097E00E946A069FC083E10E945028892B0B
:104B900009F499C080E090E00E946A0610929504A2
:104BA00092C080E090E00E946A0607CF68E024CFC0
:104BB000851709F424CF4F5F242F30E090E0F901EE
:104BC000EC5BFB4FDC01A55EBB4F7C917083F90170
:104BD000EE5EFB4F708301968F710FCF2430B1F4DE
:104BE0002091120483E194E0A5E4B4E0FC013E2F9F
:104BF000381B321718F431913D93F9CF87E3820FB8
:104C000090914404892B8093440404CF80919504AF
:104C1000823071F49160909344045E9A409A53E913
:104C2000E52E55E0F52E8E010F5F1F4FB80111C024
:104C30005E98409880910F04811103C081E08093B9
:104C40000F0480910F04833051F784E080930F04A8
:104C5000E6CFF70181917F0169A37AA30E949114A5
:104C6000F801819391938F0169A17AA1F3EAEF167C
:104C7000F5E0FF0671F780916E0545E454E087701A
:104C80000E949109CACE80915305882309F4CBCEA6
:104C90002091960431E0320F30939604291303C01B
:104CA0001092960481500E94910BBDCE10929804F0
:104CB000D8CE80917C04883011F45E9A409A89E0C5
:104CC00080937C04CECEA296ECE00C94F22C823041
:104CD000E8F4E82FF0E0EE0FFF1FEA55FA4F71837A
:104CE0006083813041F0809169008C7F842B8093B8
:104CF0006900E89A089580916900440F551F440F98
:104D0000551F837F842B80936900E99A08951F9231
:104D10000F920FB60F9211242F933F934F935F93EF
:104D20006F937F938F939F93AF93BF93EF93FF9373
:104D30008091A6059091A705892B29F0E091A60501
:104D4000F091A7050995FF91EF91BF91AF919F91C8
:104D50008F917F916F915F914F913F912F910F9024
:104D60000FBE0F901F9018951F920F920FB60F92C3
:104D700011242F933F934F935F936F937F938F9360
:104D80009F93AF93BF93EF93FF938091A80590916A
:104D9000A905892B29F0E091A805F091A9050995AD
:104DA000FF91EF91BF91AF919F918F917F916F9103
:104DB0005F914F913F912F910F900FBE0F901F90D9
:104DC00018951F920F920FB60F9211242F933F93B5
:104DD0008F939F93AF93BF938091AB059091AC0558
:104DE000A091AD05B091AE053091AA0523E0230F47
:104DF0002D3720F40196A11DB11D05C026E8230F13
:104E00000296A11DB11D2093AA058093AB05909336
:104E1000AC05A093AD05B093AE058091AF05909120
:104E2000B005A091B105B091B2050196A11DB11DCB
:104E30008093AF059093B005A093B105B093B205F0
:104E4000BF91AF919F918F913F912F910F900FBE86
:104E50000F901F9018952FB7F8946091AB05709143
:104E6000AC058091AD059091AE052FBF08953FB779
:104E7000F8948091AF059091B005A091B105B091E3
:104E8000B20526B5A89B05C02F3F19F00196A11DBC
:104E9000B11D3FBF6627782F892F9A2F620F711D92
:104EA000811D911D42E0660F771F881F991F4A954B
:104EB000D1F70895CF92DF92EF92FF92CF93DF93D5
:104EC0006B017C010E943727EB01C114D104E1047E
:104ED000F10479F00E9437276C1B7D0B683E73400C
:104EE000A0F381E0C81AD108E108F108C851DC4FED
:104EF000ECCFDF91CF91FF90EF90DF90CF900895AE
:104F0000789484B5826084BD84B5816084BD85B5A4
:104F1000826085BD85B5816085BDEEE6F0E080816B
:104F200081608083E1E8F0E010828081826080838C
:104F3000808181608083E0E8F0E08081816080830F
:104F4000E1EBF0E0808184608083E0EBF0E0808141
:104F500081608083EAE7F0E08081846080838081E3
:104F6000826080838081816080838081806880838B
:104F70001092C1000895833081F028F4813099F0B7
:104F80008230A1F008958630A9F08730B9F08430DE
:104F9000D1F4809180008F7D03C0809180008F7755
:104FA00080938000089584B58F7702C084B58F7D8B
:104FB00084BD08958091B0008F7703C08091B000C8
:104FC0008F7D8093B0000895CF93DF9390E0FC0134
:104FD000ED50F44F2491FC01E95FF34F8491882355
:104FE00049F190E0880F991FFC01E15DF34FA59115
:104FF000B4918B5D934FFC01C591D4919FB7611122
:1050000008C0F8948C91209582238C938881822308
:105010000AC0623051F4F8948C91322F309583237A
:105020008C938881822B888304C0F8948C91822B86
:105030008C939FBFDF91CF910895A1E0B0E0E3E2B0
:10504000F8E20C94DE2C282F30E0F901E152F44F05
:105050008491F901ED50F44F1491F901E95FF34F98
:1050600004910023C9F0882321F069830E94BB27A3
:105070006981E02FF0E0EE0FFF1FEB5DF34FA5918C
:10508000B4919FB7F8948C91611103C0109581235E
:1050900001C0812B8C939FBF2196E4E00C94FA2CE5
:1050A000CF93DF93282F30E0F901E152F44F849140
:1050B000F901ED50F44FD491F901E95FF34FC49138
:1050C000CC2391F081110E94BB27EC2FF0E0EE0F72
:1050D000FF1FE55EF34FA591B4912C912D2381E044
:1050E00090E021F480E002C080E090E0DF91CF9179
:1050F00008958E3008F08E50877020919D0190E4C5
:10510000299F90011124822B80937C0080917A004A
:10511000806480937A0080917A0086FDFCCF809134
:1051200078002091790090E0922B0895A0E0B0E003
:10513000ECE9F8E20C94DA2C6C017A01EB01E60E52
:10514000F71E00E010E0CE15DF0561F06991D60191
:10515000ED91FC910190F081E02DC6010995080FB9
:10516000191FF1CFC801CDB7DEB7E8E00C94F62CDB
:105170006115710589F0DB010D900020E9F7AD01A3
:1051800041505109461B570BDC01ED91FC91028007
:10519000F381E02D0995089580E090E00895EF9265
:1051A000FF920F931F93CF93DF938C01FB01C0E01D
:1051B000D0E064917F018FEFE81AF80A662361F06E
:1051C000D801ED91FC910190F081E02DC801099585
:1051D000C80FD91FF701EDCFCE01CDB7DEB7E6E09E
:1051E0000C94F82C0E94B8280895DC01ED91FC91F4
:1051F0000190F081E02D099508950F931F93CF93AF
:10520000DF93EC016DE00E94F5288C016AE0CE018D
:105210000E94F528800F911FDF91CF911F910F9170
:1052200008950F931F93CF93DF93EC010E94CF2833
:105230008C01CE010E94FD28800F911FDF91CF913C
:105240001F910F9108950F931F93CF93DF93EC015C
:105250000E94B8288C01CE010E94FD28800F911F6A
:10526000DF91CF911F910F9108950F931F93CF93CB
:10527000DF93EC010E94F5288C01CE010E94FD28ED
:10528000800F911FDF91CF911F910F910895A1E29F
:10529000B0E0EDE4F9E20C94D62C7C01C42EE52FAD
:1052A000CB01D22E19A221E02D1510F02AE0D22E2A
:1052B0008E010F5D1F4F8D2C912CA12CB12C6C2DCC
:1052C0007E2FA50194010E948F2C8C2DD29E8019D7
:1052D0001124015011098A3010F4805D01C0895CED
:1052E000F8018083211531054105510521F0C22EB9
:1052F000E32FCA01E4CFB801C7010E94B828A196E4
:10530000ECE00C94F22CA0E0B0E0E9E8F9E20C94B7
:10531000DA2CEC016A017B012115310541F4E881A9
:10532000F9810190F081E02D642F09951DC02A308C
:105330003105A9F477FF12C06DE20E94F5288C01B7
:1053400044275527BA014C195D096E097F092AE0E7
:10535000CE010E944729800F911F06C02AE0B701A5
:10536000A601CE010E944729CDB7DEB7E8E00C9434
:10537000F62C9A01AB01662757FD6095762F0E94A7
:10538000832908950F931F93CF93DF93EC019A0124
:10539000AB01662757FD6095762F0E9483298C010B
:1053A000CE010E94FD28800F911FDF91CF911F91A8
:1053B0000F9108952115310549F4DC01ED91FC911F
:1053C0000190F081E02D642F099508950E944729EE
:1053D00008959A01462F50E060E070E00E94DA29BB
:1053E00008959A01AB0160E070E00E94DA29089507
:1053F0000F931F93CF93DF93EC010E94DA298C0166
:10540000CE010E94FD28800F911FDF91CF911F9147
:105410000F9108950F931F93CF93DF93EC019A019F
:10542000AB0160E070E00E94DA298C01CE010E949D
:10543000FD28800F911FDF91CF911F910F9108954B
:105440000F931F93CF93DF93EC019A01462F50E007
:1054500060E070E00E94DA298C01CE010E94FD28F4
:10546000800F911FDF91CF911F910F910895FC0143
:1054700024853585F901E05CFF4F80819181F90138
:10548000EE5BFF4F20813181821B930B8F73992735
:105490000895FC0184859585FC01E05CFF4F408107
:1054A0005181FC01EE5BFF4F208131814217530790
:1054B00041F00190F081E02DE80FF91F808190E02C
:1054C00008958FEF9FEF0895FC0184859585FC0179
:1054D000E05CFF4F40815181FC01EE5BFF4F20817A
:1054E00031814217530779F0A081B181A80FB91F0C
:1054F0008C91208131812F5F3F4F2F733327318370
:10550000208390E008958FEF9FEF0895FC0181A123
:10551000882329F0A489B5898C9186FFFBCF11A23D
:105520000895CF93DF93FC0126853785D901A05CD0
:10553000BF4F8D919C91119701968F739927E90127
:10554000CE5BDF4F4881598184179507D9F30D90C1
:10555000BC91A02DA20FB31F6C93A685B785A05C4C
:10556000BF4F11969C938E93A689B7892C9181E0A9
:1055700090E0078C02C0880F991F0A94E2F7282B4D
:105580002C9381E081A30488F589E02D80818064DB
:10559000808381E090E0DF91CF91089508951F927C
:1055A0000F920FB60F9211242F933F934F938F9327
:1055B0009F93EF93FF938091C00082FD1CC04091A8
:1055C000C6008091590690915A0601968F739927CB
:1055D00020915B0630915C068217930771F0E09191
:1055E0005906F0915A06E75EF94F408390935A06A8
:1055F0008093590602C08091C600FF91EF919F9160
:105600008F914F913F912F910F900FBE0F901F9050
:10561000189583EB95E00E94372A892B11F00E94A0
:10562000CE2A08951F920F920FB60F9211242F9336
:105630003F938F939F93EF93FF93209115063091A3
:10564000160680911706909118062817390731F42D
:105650008091C1008F7D8093C10014C0E091170636
:10566000F0911806EB52FA4F208180911706909125
:10567000180601968F739927909318068093170642
:105680002093C600FF91EF919F918F913F912F91B1
:105690000F900FBE0F901F901895A0E0B0E0E3E5CB
:1056A000FBE20C94D62CFC011382128288EE93E06C
:1056B000A0E0B0E084839583A683B7838EE893E06F
:1056C000918380837587648757874687318B208BCA
:1056D000138B028BF58AE48AD78AC68AB18EA08E94
:1056E000938E828E8F85848F8889858F8989868F16
:1056F0008A89878F8B8980A3ECE00C94F22CCF925F
:10570000DF92EF92FF92CF93DF93EC016A017B016E
:10571000411581EE580761057105F9F0EC89FD89A5
:1057200081E090E008A002C0880F991F0A94E2F778
:10573000808360E079E08DE390E0A70196010E940C
:105740008F2C2150310941095109569547953795BC
:105750002795211580E1380798F0EC89FD891082A2
:1057600060E874E88EE190E0A70196010E948F2C1A
:10577000215031094109510956954795379527958B
:10578000E889F9893083EA89FB89208319A2EE89A7
:10579000FF89408181E090E09C010C8C02C0220FC7
:1057A000331F0A94E2F7422B4083EE89FF89408140
:1057B0009C010D8C02C0220F331F0A94E2F7422B8A
:1057C0004083EE89FF8940819C010E8C02C0220F2C
:1057D000331F0A94E2F7422B4083EE89FF89208130
:1057E0000F8C02C0880F991F0A94E2F780958223DC
:1057F0008083DF91CF91FF90EF90DF90CF9008955D
:105800008F929F92AF92BF92CF92DF92EF92FF92D0
:105810000F931F9381E08F9385E08F9387E08F93A1
:1058200083E08F9384E08F93E6EC8E2E912CF2EC44
:10583000AF2EB12CA1ECCA2ED12CB0ECEB2EF12C5A
:1058400004EC10E025EC30E045ED55E069E176E050
:1058500083EB95E00E944D2B0F900F900F900F90CF
:105860000F901F910F91FF90EF90DF90CF90BF901E
:10587000AF909F908F9008950E9480270E94E22011
:10588000C9E0DBE20E9480232097E1F30E94092B0C
:10589000F9CFA29FB001B39FC001A39F700D811DDE
:1058A0001124911DB29F700D811D1124911D089529
:1058B0000E94492CA59F900DB49F900DA49F800D30
:1058C000911D11240895B7FF0C94582C0E94582C58
:1058D000821B930B0895DB018F939F930E94582C9A
:1058E000BF91AF91A29F800D911DA39F900DB29F7C
:1058F000900D1124089597FB072E16F4009407D0FD
:1059000077FD09D00E940D2D07FC05D03EF490953F
:1059100081959F4F0895709561957F4F0895A1E2FD
:105920001A2EAA1BBB1BFD010DC0AA1FBB1FEE1F19
:10593000FF1FA217B307E407F50720F0A21BB30B64
:10594000E40BF50B661F771F881F991F1A9469F7E0
:1059500060957095809590959B01AC01BD01CF013C
:105960000895052E97FB1EF400940E94C82C57FD45
:1059700007D00E948F2C07FC03D04EF40C94C82C47
:1059800050954095309521953F4F4F4F5F4F08956B
:1059900090958095709561957F4F8F4F9F4F08959B
:1059A0002F923F924F925F926F927F928F929F922F
:1059B000AF92BF92CF92DF92EF92FF920F931F931D
:1059C000CF93DF93CDB7DEB7CA1BDB0B0FB6F894CE
:1059D000DEBF0FBECDBF09942A88398848885F840E
:1059E0006E847D848C849B84AA84B984C884DF807F
:1059F000EE80FD800C811B81AA81B981CE0FD11D63
:105A00000FB6F894DEBF0FBECDBFED010895EE0FC7
:105A1000FF1F0590F491E02D0994AA1BBB1B51E1D7
:105A200007C0AA1FBB1FA617B70710F0A61BB70B0E
:105A3000881F991F5A95A9F780959095BC01CD01B3
:105A400008958F929F92AF92BF92CF92DF92EF9282
:105A5000FF92CF93DF93EC01688179818A819B81EA
:105A6000611571058105910521F464E279ED8BE5FD
:105A700097E02DE133EF41E050E00E94B12C490165
:105A80005A019B01AC01A7EAB1E40E94582C6B01BA
:105A90007C01ACEEB4EFA50194010E94662CC60E09
:105AA000D71EE81EF91EF7FE06C081E0C81AD1080D
:105AB000E10880E8F80AC882D982EA82FB82C7013D
:105AC000B6019F77DF91CF91FF90EF90DF90CF905D
:105AD000BF90AF909F908F9008950E94212D0895C0
:105AE00086E091E00E94212D089560930601709355
:105AF0000701809308019093090108952F923F9226
:105B00005F926F927F928F929F92AF92BF92CF924D
:105B1000DF92EF92FF920F931F93CF93DF938B014E
:105B2000EA016115710521F0DB018C9311969C93BC
:105B3000209739F09E01225031092332310508F0B7
:105B4000D8C07C016701BFEFCB1ADB0A5601F70111
:105B50006080862D90E00E94B02E892B11F0760196
:105B6000F1CFFDE26F120AC0570182E0A80EB11C0E
:105B7000D70111966C90772473940BC0BBE26B1223
:105B800007C05701E2E0AE0EB11CD70111966C9030
:105B9000712CCE018F7E892B89F4B0E36B1237C054
:105BA000F50180818F7D8835D1F46180F2E0AF0E00
:105BB000B11C872D8260782EC0E1D0E0CA30D105BB
:105BC00051F1C031D10521F0C830D10599F409C097
:105BD000CC24CA94DC2CEC2CAFE0FA2E22C0209707
:105BE00069F7C8E0D0E0CC24CA94DC2CEC2CFFE1AF
:105BF000FF2E17C06FEF7FEFCB019E01442737FDCB
:105C00004095542F0E948F2C69017A010AC0209779
:105C1000A9F6CAE0D0E0E9E9CE2EDC2CEC2CE9E1D3
:105C2000FE2EF50160E020E030E0A9014E01AA243B
:105C300097FCA094BA2C1F0170ED572E560CA9E0CA
:105C4000A51570F48FEB860D8A3118F499EC592E56
:105C500006C08FE9860D8A3148F589EA582E560C20
:105C6000852D90E08C179D070CF56F3FD9F0C2167B
:105C7000D306E406F50698F0C501B4010E946B2C2A
:105C80009B01AC01852D90E0A0E0B0E0280F391F0A
:105C90004A1F5B1F281739074A075B0710F46FEF8D
:105CA00001C061E03196D1016C90C5CF011511059D
:105CB00051F0662311F0319703C071FE04C0329792
:105CC000D801ED93FC9370FE07C050954095309538
:105CD00021953F4F4F4F5F4F67FF10C082E290E02A
:105CE00090935E0680935D066FEF7FEF8FEF9FEFDF
:105CF00007C060E070E080E090E002C0B901CA0136
:105D0000DF91CF911F910F91FF90EF90DF90CF9097
:105D1000BF90AF909F908F907F906F905F903F90DB
:105D20002F900895FC0188279927E894219120322B
:105D3000E9F3293010F02E30C8F32B3241F02D3228
:105D400039F4689404C00E94E42E820F911D2191C1
:105D500020532A30C0F31EF4909581959F4F0895EB
:105D6000911150C0803219F089508550D0F70895B4
:105D70004AE953E00E94BD2E0895FA01A191B08135
:105D8000009719F41097E1F0CD01DC01CD010D90E1
:105D9000002011F4C00113C0FB012191222319F04E
:105DA0002015D9F7F3CFFB012191201519F41E928C
:105DB000119606C02223C1F70D900020A1F7D00153
:105DC000FA01A193B08308957AE0979F902D879F61
:105DD000802D910D11240895F999FECF92BD81BDBA
:105DE000F89A992780B50895262FF999FECF1FBA02
:105DF00092BD81BD20BD0FB6F894FA9AF99A0FBEF4
:0E5E000001960895992788270895F894FFCFFA
:105E0E0000005F06200001000000FF0002000200FB
:105E1E000200020002000200020002000200020064
:105E2E0002000200020002000200028025000005AE
:105E3E00400AA1204EA50020244EA52C2330C012CE
:105E4E0000001A400AA1204EA5001B1E27522C232B
:105E5E00308025000005400AA1204EA50020244ECA
:105E6E00A52C2330004B000006400AD0009D4900AF
:105E7E007B289D492C233000E1000005400A450196
:105E8E00D7DC03B81E0EBF00232E48E801008A405F
:105E9E000A6001555502AD1E20000023C80154585A
:105EAE002074696D656F75742100596573004E6FAE
:105EBE00002C00386368004E2F41002C205B005DE3
:105ECE002028002900486F70206368616E6E656C33
:105EDE002000204020007363616E6E6572206D6F2E
:105EEE006465004E4F5420454E41424C454400538C
:105EFE00656E64696E672073657474696E6773206E
:105F0E00746F2052580A00526573657474696E6717
:105F1E002073657474696E6773206F6E2052580A11
:105F2E000041626F727465642065646974730A005F
:105F3E00696E76616C69642073656C656374696FF4
:105F4E006E000D0A496E76616C696420696E70751B
:105F5E0074202D2064697363617264656421070087
:105F6E0053657474696E677320736176656420740B
:105F7E006F20454550524F4D0A005265766572743A
:105F8E0065642073657474696E67732066726F6DD5
:105F9E0020454550524F4D0A004C6F616465642098
:105FAE00666163746F72792064656661756C747373
:105FBE000A004B657920616E64206368616E6E65C0
:105FCE006C732072616E646F6D697A65640A004F3E
:105FDE0070656E4C52536E67205458207374617204
:105FEE0074696E672000206F6E20485720006D6F19
:105FFE0064756C65206C6F636B65643F00342B3485
:10600E00003800382B340031320031322B3400315D
:10601E00360050504D0052535349005344410053E3
:10602E00434C00525844005458440041494E004CD1
:10603E00424545500053504B54524D005342555318
:10604E000053554D44004C4C494E440000070B0C78
:10605E0010111500B701FD020103030307030A0324
:10606E000F03B701160A13223129120316031B035D
:10607E001F03230327032B032F0335033C03410385
:10608E0046035F025F025F025F0200000000912A7A
:0A609E009628372A642A492A862A28
:107E00000F92CDB7DEB7112484B714BE81FFF1D035
:107E100082E08093C00088E18093C10086E0809377
:107E2000C20080E18093C4008EE0CDD088249924E4
:107E3000CC24C394F5E0DF2EE1E1EE2E73E0F72EC3
:107E4000B6D0082F813479F4B2D08983C2D0898129
:107E5000823811F481E005C0813811F485E001C059
:107E600083E09ED09AC0823411F484E103C085344B
:107E700019F485E0B6D091C0853561F498D0082F0B
:107E800010E095D090E0982E8824802A912A880CC2
:107E9000991C82C0863521F484E0A3D080E0E1CF34
:107EA000843609F04CC083D082D0A82E80D0B82E62
:107EB00000E011E07CD0F80181938F01AE16D1F77C
:107EC00088D0FB2DF53489F4E0E0F1E00BC0F9999E
:107ED000FECF92BC81BC0894811C911C819180BD15
:107EE000FA9AF99AEA1598F358C08B2D863409F05E
:107EF00054C0F401F7BEE89507B600FCFDCFF401CD
:107F0000A0E0B1E02C9130E011968C91119790E0B7
:107F1000982F8827822B932B12960C01C7BEE895C9
:107F20001124329681E0A038B80761F7F401D7BE7A
:107F3000E89507B600FCFDCFE7BEE8952EC0843774
:107F4000F1F435D034D0182F32D0B82E42D0FB2DDA
:107F5000F63421F4F40105914F010CC0FB2DF534EA
:107F600049F4F999FECF92BC81BC0894811C911C04
:107F7000F89A00B5802F14D0115049F70EC08537FC
:107F800039F427D08EE10CD085E90AD08FE069CF93
:107F9000813511F488E017D01CD080E101D050CF9A
:107FA0009091C00095FFFCCF8093C600089580910A
:107FB000C00087FFFCCF8091C00084FD01C0A89560
:107FC0008091C6000895E0E6F0E098E19083808318
:107FD0000895EDDF803219F088E0F5DFFFCF84E10E
:107FE000DFCF1F93182FE3DF1150E9F7F2DF1F9166
:0E7FF0000895282E80E0E7DFEE27FF27099492
:027FFE0001057B
:0400000300007E007B
:00000001FF
